:100000000C9470060C94A8060C94A8060C94A806F0
:100010000C94A8060C94A8060C94A8060C94A806A8
:100020000C94A8060C94A8060C944B2B0C941D2C35
:100030000C946C250C94A8060C94A8060C94A806A5
:100040000C94A8060C94A8060C94A8060C94A80678
:100050000C94A8060C94F4250C94A8060C94A806FD
:100060000C94A8060C94A8060C94A8060C94A80658
:100070000C94A8060C94A8060C94A8060C94A80648
:100080000C94A8060C94A8060C94A8060C94A80638
:100090000C94A8060C94A8060C94A8060C94A80628
:1000A0000C94A8060C94A8060C94A806820A820A4E
:1000B000AE0AAE0A160B340B4C0C4C0C3F0BD80B93
:1000C000E90BE90B99218721A021F6204D224D2231
:1000D00084214D224D22CD214D22E1212D224D2280
:1000E0004D224D224D2201224D224D22FE214D2234
:1000F000B9214D224D22472247224722472247223B
:10010000472247224722472249224D2299217C211A
:100110004D224D224D224D224D224D224D224D2267
:100120004D224D2249224D224D2284214D2245222D
:100130004522452245224522452245224522452287
:1001400049228A2CB12CA92DB12CA92DFD2C202DB2
:10015000A92D772D862D29001E001F0020002100CB
:100160002200230024002500260027002D002E0059
:100170002A002B0014001A000800150017001C00AC
:1001800018000C00120013002F003000310039005D
:1001900004001600070009000A000B000D000E0005
:1001A0000F003300340028000000E10000001D00B3
:1001B0001B00060019000500110010003600370072
:1001C000387252000100E000E300E2000000280065
:1001D00001512C000000E600E400500051004F00E7
:1001E0000000010001000100010001000100010008
:1001F00001000100010001000100010001000100F7
:1002000001000100010001000100010001000100E6
:1002100001000100010001000100010001000100D6
:1002200001000100010001000100010001000100C6
:1002300001000100000001000000010001000100B8
:1002400001000100010001000100010001000100A6
:100250000100010001000100000001000100010097
:100260000000010001000100010001000000444500
:100270004255473A2064697361626C65642E0A00D6
:1002800044454255473A20656E61626C65642E0AAA
:10029000000A0025303258006C65645F7461736B2E
:1002A0003A20004F6E6573686F743A206163746919
:1002B00076653A2025640A000A002530313662004E
:1002C0003A200025303258000A722F632030313234
:1002D000333435363738394142434445460A0029DC
:1002E0000A002575002F002575005D280025640093
:1002F0002000256400200025640020002564007C87
:100300000025303258006D6F7573656B6579205B21
:1003100062746E7C782079207620685D2872657022
:100320002F61636C293A205B006261636B6C6967C3
:10033000687420737465703A2025750A00626163E1
:100340006B6C696768742064697361626C650A002C
:100350006261636B6C6967687420656E61626C656D
:100360000A006261636B6C6967687420746F676709
:100370006C653A2025750A006261636B6C69676879
:10038000742064656372656173653A2025750A009F
:100390006261636B6C6967687420696E6372656122
:1003A00073653A2025750A00313A0964656C6179F4
:1003B000282A31306D73293A2025750A323A0969A5
:1003C0006E74657276616C286D73293A2025750A02
:1003D000333A096D61785F73706565643A202575FD
:1003E0000A343A0974696D655F746F5F6D61783ABC
:1003F0002025750A353A09776865656C5F6D617807
:100400005F73706565643A2025750A363A09776826
:1004100065656C5F74696D655F746F5F6D61783A77
:100420002025750A00703A097072696E7420766131
:100430006C7565730A643A09736574206465666156
:10044000756C74730A75703A092B310A646E3A0937
:100450002D310A6C743A092B31300A72743A092D25
:1004600031300A4553432F713A09717569740A0A8C
:100470007370656564203D2064656C7461202A207A
:100480006D61785F7370656564202A2028726570DD
:10049000656174202F2074696D655F746F5F6D6195
:1004A00078290A77686572652064656C74613A2002
:1004B000637572736F723D25642C20776865656C77
:1004C0003D25640A53656520687474703A2F2F6562
:1004D0006E2E77696B6970656469612E6F72672F24
:1004E00077696B692F4D6F7573655F6B6579730AFB
:1004F000004D3E20004D25753A25733E20003F0AF1
:10050000003D2025750A003F0A0064656661756C30
:1005100074730A0025750A003F0A000A092D205647
:10052000616C756573202D0A00710A000A092D207F
:100530004D6F7573656B6579202D0A003F00433E52
:1005400020004C25640A000A092D2053746174753B
:1005500073202D0A686F73745F6B6579626F6172C7
:10056000645F6C65647328293A20253032580A6B21
:100570006579626F6172645F70726F746F636F6CC4
:100580003A20253032580A6B6579626F6172645F78
:1005900069646C653A20253032580A6B65796D6163
:1005A000705F636F6E6669672E6E6B726F3A20259F
:1005B0003032580A74696D65725F726561643332F6
:1005C00028293A202530386C580A000A092D20566F
:1005D000657273696F6E202D0A5649443A2030784F
:1005E000464541452854686556616E204B657962E1
:1005F0006F6172647329205049443A20307838384A
:1006000037302842616E616E6153706C69742036B8
:100610003029205645523A203078303030310A4265
:1006200055494C443A202028466562203238203211
:10063000303232290A4F5054494F4E533A204C55CC
:100640004641204D4F5553454B455920455854522E
:10065000414B455920434F4E534F4C4520434F4D3E
:100660004D414E44204E4B524F20343039360A47CC
:1006700043433A20352E342E30204156522D4C49DA
:1006800042433A20322E302E30204156525F4152A2
:1006900043483A20617672350A000A092D20436FDB
:1006A0006E736F6C65202D0A4553432F713A0971A3
:1006B0007569740A6D3A096D6F7573656B65790AB2
:1006C000000A092D204D61676963202D0A443A090B
:1006D0004465627567204D65737361676520546F6B
:1006E00067676C650A583A094D61747269782044ED
:1006F00065627567204D6F646520546F67676C6530
:10070000202D2053686F77206B6579707265737345
:10071000657320696E206D617472697820677269F3
:10072000640A4B3A094B6579626F617264204465D3
:1007300062756720546F67676C65202D2053686F62
:1007400077206B65797072657373207265706F7254
:10075000740A4D3A094465627567204D6F7573657B
:1007600020546F67676C650A563A0956657273695B
:100770006F6E0A533A095374617475730A433A09E8
:10078000416374697661746520436F6E736F6C6545
:10079000204D6F64650A46312D4631303A09537752
:1007A0006974636820746F204C6179657220302D04
:1007B000392028463130203D204C30290A302D394F
:1007C0003A0953776974636820746F204C617965C6
:1007D0007220302D390A47524156453A09537769FC
:1007E00074636820746F204C617965722030202812
:1007F000616C7465726E617465290A423A094A75C2
:100800006D7020746F20426F6F746C6F61646572DD
:100810000A4553433A094A756D7020746F20426F40
:100820006F746C6F616465722028616C7465726EA0
:10083000617465290A453A095072696E742045450C
:1008400050524F4D2053657474696E67730A42535A
:10085000504143453A09436C656172204545505209
:100860004F4D0A4E3A094E4B524F20546F67676CFA
:10087000650A006261636B6C696768745F636F6EC1
:100880006669672E7261773A20253032580A2E65E4
:100890006E61626C653A2025750A2E6C6576656C12
:1008A0003A2025750A006B65796D61705F636F6E24
:1008B0006669672E7261773A20253032580A2E73A6
:1008C0007761705F636F6E74726F6C5F636170737A
:1008D0006C6F636B3A2025750A2E636170736C6FC1
:1008E000636B5F746F5F636F6E74726F6C3A202519
:1008F000750A2E737761705F6C63746C5F6C6775DB
:10090000693A2025750A2E737761705F7263746C83
:100910005F726775693A2025750A2E737761705F7B
:100920006C616C745F6C6775693A2025750A2E736B
:100930007761705F72616C745F726775693A2025C8
:10094000750A2E6E6F5F6775693A2025750A2E73DA
:100950007761705F67726176655F6573633A2025C2
:10096000750A2E737761705F6261636B736C61737C
:10097000685F6261636B73706163653A2025750A15
:100980002E6E6B726F3A2025750A0064656275677A
:100990005F636F6E6669672E7261773A2025303229
:1009A000580A2E656E61626C653A2025750A2E6DB7
:1009B00061747269783A2025750A2E6B6579626FC9
:1009C0006172643A2025750A2E6D6F7573653A2041
:1009D00025750A006565636F6E6669673A0A646526
:1009E0006661756C745F6C617965723A2025750A71
:1009F000003F004E4B524F3A206F66660A004E4B46
:100A0000524F3A206F6E0A000A6D6F7573653A2077
:100A10006F66660A000A6D6F7573653A206F6E0A1D
:100A2000000A6B6579626F6172643A206F66660ACC
:100A3000000A6B6579626F6172643A206F6E0A001A
:100A40000A6D61747269783A206F66660A000A6DF1
:100A500061747269783A206F6E0A000A6465627583
:100A6000673A206F66660A000A64656275673A2015
:100A70006F6E0A000A0A4A756D70696E6720746F9E
:100A800020626F6F746C6F616465722E2E2E200071
:100A9000433E2000436C656172696E672045455096
:100AA000524F4D0A000A002530325820006B6579FC
:100AB000626F6172645F7265706F72743A20006475
:100AC000656C5F6B65795F6269743A2063616E275C
:100AD000742064656C3A20253032580A00616464E1
:100AE0005F6B65795F6269743A2063616E27742079
:100AF0006164643A20253032580A005B735D005B04
:100B0000575D005B535D005B525D005B445D005BC5
:100B1000435D001E03420061006E0061006E0061D3
:100B200000530070006C0069007400200036003033
:100B30000000002203540068006500560061006E4A
:100B40000020004B006500790062006F00610072B8
:100B5000006400730000000403090409025B000341
:100B60000100A0FA0904000001030101000921119C
:100B7000010001224000070581030800010904016A
:100B800000010300000009211101000122B6000745
:100B9000058203200001090402000203000000098D
:100BA0002111010001222200070583032000010713
:100BB0000503032000011201000200000008AEFE40
:100BC00070880100010200010631FF0974A10109CA
:100BD00075150026FF00952075088102097615001D
:100BE00026FF00952075089102C005010902A101A8
:100BF00085020901A100050919012908150025012F
:100C00009508750181020501093009311581257F9B
:100C100095027508810609381581257F95017508AB
:100C20008106050C0A38021581257F95017508811A
:100C300006C0C005010980A101850319012AB7007A
:100C4000150126B700950175108100C0050C09013A
:100C5000A101850419012AA002150126A00295010F
:100C600075108100C005010906A101850605071957
:100C7000E029E7150025019508750181020507198E
:100C80000029EF1500250195F0750181020508196D
:100C9000012905950575019102950175039101C022
:100CA00005010906A101050719E029E7150025013D
:100CB00095087501810295017508810105071900E4
:100CC00029FF150026FF0095067508810005081903
:100CD000012905950575019102950175039101C0E2
:100CE00011241FBECFEFDAE0DEBFCDBF04B603FE96
:100CF00018C08091340390913503A0913603B091D0
:100D000037038730904BA740B04B59F4109234030F
:100D1000109235031092360310923703E0E0F8E3A7
:100D2000099511E0A0E0B1E0E6E6FDE502C005901E
:100D30000D92AA3FB107D9F723E0AAEFB1E001C0B5
:100D40001D92A433B207E1F70E94CB180C94B12E88
:100D50000C940000FF93EF93E091FA01F091FB01F6
:100D6000309709F00995EF91FF910895FC01859165
:100D7000803011F0EFDFFBCF0895FF27E0E230E293
:100D800047FF0CC0419597FF09C0EDE26095709553
:100D900080959095611D711D811D911D27FF02C0D9
:100DA000219530E350E2AA27660F771F881F991F0D
:100DB000AA1FA41710F0A41B63955A95A9F7AA308F
:100DC00008F0A95FA05DAF93F395611571058105EA
:100DD000910541F7ED3211F4EF93F395F21718F402
:100DE0003F93F395FBCF8F91B5DFFA95E1F7089527
:100DF000E991F9918591803021F0853219F0AADFCF
:100E0000F9CF089520E0E89455915532C1F350335D
:100E100011F4689455915A3348F4505390F3220FCB
:100E2000022E220F220F200D250FF4CF0EF4219554
:100E300089919991533619F3533729F1533559F163
:100E4000BC0188279927E8945C3621F4899199910F
:100E500068945591543639F446EF7EF077FF0DC013
:100E60008FEF9FEF0AC055374AE039F0583540E11F
:100E700021F0523642E009F00895FF93EF937DDFB1
:100E8000EF91FF91B7CFFF93EF93FC0181918030F9
:100E9000B9F360DFFBCFFF93EF9368DFF1CFDF9310
:100EA000CF93CDB7DEB72596A3DFCF91DF9108951D
:100EB00081E0089581E008950C945A0708950C94F8
:100EC0005E071F93CF93DF9300D000D01F92CDB762
:100ED000DEB749835A836B833091FD0189819A8102
:100EE000311114C0662359F0222349F00E94890E63
:100EF000182F682F89819A810E94320E03C00E94A8
:100F00005D0E182F69817A81812F04C00E94890E9D
:100F100069817A810F900F900F900F900F90DF9161
:100F2000CF911F910C94D915FC01262F408151813E
:100F30006281738184810C94610781E00895CF936D
:100F4000DF93EC0160E00E949407BE01DF91CF9136
:100F50000C945F070C9463170C945F1708950E941C
:100F6000DC0C0E94AE072FEF84E39CE02150804010
:100F70009040E1F700C000000C941A260F931F93D5
:100F8000CF93DF938C0161E00E949407EC01B801DC
:100F90000E945C07882309F462C0B801CE010E9458
:100FA0003C1D882309F45BC0B801CE010E945A237E
:100FB000882309F454C0B801CE010E94371E88234B
:100FC00009F44DC0B801CE010E94B622882309F46D
:100FD00046C0F80182818823D9F1CF3D8CE5D8073E
:100FE00079F140F4C115FCE5DF0791F0C130DC4533
:100FF00091F02EC0CC35EDE5DE0741F1CD35FDE5B4
:10100000DF0709F1CB35DD4519F50E94201320C01B
:101010000E94AF0724C08091C102C82FC095C17043
:10102000C0FB80F98093C102CC2329F080E892E0D4
:101030000E94B60614C08EE692E00E94B60610C06A
:101040000E94D4130CC00E94171302C00E942313E5
:10105000C801DF91CF911F910F910C945807C0E008
:101060008C2FDF91CF911F910F9108950E944E25F3
:1010700080E00E94711D0C9479080E94F41B0E946C
:101080007C080C9454258295982F937344E0949F88
:10109000900111248C7C86958695282B822F85754E
:1010A000880F2A7A2695822B0895CF93DF93D92F24
:1010B0000E944308C82F8D2F0E9443082C2F30E038
:1010C000322F2227A901482BCA01DF91CF91089521
:1010D00008950C94680881E008950C946B080895B5
:1010E000CF93C82F0E9469088C2F0E946D08CF9162
:1010F000089580E00C9470080E94B6230C94700848
:10110000CF930E94B623C82F8091FC01C81741F1EC
:10111000C093FC018091C10282FF1EC080FF04C009
:1011200088E992E00E94B6068091C10280FF0CC05F
:101130001F92CF9383E992E09F938F930E944F0772
:101140000F900F900F900F908091C10280FF04C00C
:1011500081E992E00E94B6068C2FCF910C94700822
:10116000CF910895CF93DF93CDB7DEB72B970FB60E
:10117000F894DEBF0FBECDBF4F83588769877A874B
:101180008B8761110E944F129E012F5F3F4F86E0B7
:10119000F90111928A95E9F785E0FE013796D901A8
:1011A00001900D928A95E1F789819A814C815D8148
:1011B000452B31F09F3F31F491E08F3F19F403C08C
:1011C00091E001C090E090FF09C049815A816B8194
:1011D0007C818D819E810E94701105C0C9010E9491
:1011E0009D078111F2CF2B960FB6F894DEBF0FBE8C
:1011F000CDBFDF91CF910895FC01808191810E9444
:10120000CB0E0895CF93882309F4A9C0C82F823844
:10121000C1F40E94B62381FDA2C069E3809102015E
:10122000909103010E9409250E9471122FEF81EE17
:1012300094E0215080409040E1F700C0000069E355
:1012400019C0833801F50E94B62380FD88C063E58C
:1012500080910201909103010E9409250E94711260
:101260002FEF81EE94E0215080409040E1F700C0E4
:10127000000063E580910201909103010E94142512
:10128000CF910C9471128438C1F40E94B62382FD70
:1012900066C067E480910201909103010E940925D4
:1012A0000E9471122FEF81EE94E021508040904017
:1012B000E1F700C0000067E4DDCF8CEF8C0F813ACE
:1012C000F8F48C2F0E945F22811149C06C2F80910D
:1012D0000201909103010E946724882349F06C2F3A
:1012E00080910201909103010E9414250E947112C5
:1012F0006C2F80910201909103010E940925C0CFBB
:1013000080E28C0F883048F4C77081E001C0880FFC
:10131000CA95EAF70E943212B3CFEBE5EC0FE33047
:1013200040F4F0E0E95BFE4F808190E0CF910C94B7
:101330002524E8E5EC0FE73150F4F0E0EE0FFF1F55
:10134000E75EFE4F80819181CF910C943B24CD3E8E
:1013500030F08C2F0E945019CF910C94221ACF910B
:101360000895882309F464C0823879F40E94B62372
:1013700081FF5EC069E380910201909103010E94A8
:1013800009250E94711269E310C08338B1F40E94EC
:10139000B62380FF4DC063E5809102019091030167
:1013A0000E9409250E94711263E5809102019091CB
:1013B00003010E9414250C947112843879F40E9460
:1013C000B62382FF35C067E480910201909103014A
:1013D0000E9409250E94711267E4E7CF9CEF980FE5
:1013E000913A10F4682FE1CF90E2980F983050F4C2
:1013F000877091E001C0990F8A95EAF7892F0E94C2
:101400003812D9CF9BE5980F933020F480E090E01C
:101410000C94252498E5980F973120F480E090E013
:101420000C943B248D3E20F00E94AB190C94221AA0
:1014300008951F93CF93DF93182FEB010E940209A9
:10144000209741F08FE99FE00197F1F700C000007D
:101450002197F6CF812FDF91CF911F910C94B10985
:10146000893319F060E070E002C060E570E00C9430
:10147000190A882321F00E9432120C9471120895E7
:10148000882321F00E9438120C9471120895CF9293
:10149000DF92EF92FF920F931F93CF93DF937C0124
:1014A000D62FC72FFC011281058102950F700E9473
:1014B00028128823B9F01123A9F08C2F807F803463
:1014C00021F080E28D0F883068F080910D0382FD5D
:1014D00009C082E00E94D1120E94281291E0D82E09
:1014E000D92601C0D12CCC2EC2948FE0C8228C2DDD
:1014F00090E08C30910508F0CFC1FC01EA5AFF4F13
:101500000C94422E8C2F807FCF70882311F0C295CF
:10151000C07F112399F0CC2309F4AAC180E28D0F7A
:10152000883010F0D11104C08C2F0E94321203C0F9
:101530008C2F0E9442120E9471129AC18D2F0E941C
:10154000B109CC2309F4A8C180E28D0F883038F1AD
:10155000DD2329F18C2F0E94481224C08C2F807F1C
:10156000CF70803211F0C295C07FDD2319F0D130E9
:10157000A1F13DC080910D0382FF17C0112349F0F6
:10158000CC2329F08C2F0E9432120E94711280E02D
:1015900070C180E00E94B109CC2309F47DC18C2F79
:1015A0000E9438120E94711277C1112371F000233A
:1015B00041F0013031F40E9452128C2B0E945A12D9
:1015C0006BC10E9452128C2B1DC0002319F00130F8
:1015D00009F462C10E94671225C0112321F0063070
:1015E00008F05AC10EC0053008F056C11BC01123C7
:1015F00061F0002331F0F701858180FF39C18F70E0
:1016000085838C2F0E94390A47C1002359F0D933B2
:1016100009F03FC1FFEF07EE13E0F150004010402A
:10162000E1F735C18C2F0E94400A36C18C2F869578
:101630008695837019F0813061F02EC1112321F05D
:101640008D2F9C2F937002C080E090E00E94252493
:101650002BC1112321F08D2F9C2F937002C080E0AD
:1016600090E00E943B2420C18D2F112319F00E948D
:10167000501902C00E94AB190E94221A15C18C2F6A
:10168000837009F047C011110BC12D2F22952695AB
:101690002770220F220F6D2F6F70862F90E0A0E031
:1016A000B0E0022E04C0880F991FAA1FBB1F0A9426
:1016B000D2F7D4FF10C04FE050E060E070E004C00B
:1016C000440F551F661F771F2A95D2F740955095F6
:1016D0006095709503C040E050E0BA01C695C6958C
:1016E000C3708A019B01082B192B2A2B3B2BC901A4
:1016F000B801C23049F058F4C13019F00E94480DC9
:10170000CFC00E94360DCCC00E945A0DC9C00E94A5
:10171000340DC6C0112319F08C2F817001C086953D
:10172000882309F4BDC02D2F229526952770220FFE
:10173000220F6D2F6F70862F90E0A0E0B0E0022E98
:1017400004C0880F991FAA1FBB1F0A94D2F7D4FFA9
:1017500010C04FE050E060E070E004C0440F551F3F
:10176000661F771F2A95D2F7409550956095709522
:1017700003C040E050E0BA01C695C695C3708A0127
:101780009B01082B192B2A2B3B2BC901B801C23016
:1017900049F058F4C13019F00E940D0E81C00E942A
:1017A000FB0D7EC00E941F0E7BC00E946E0D78C094
:1017B000CF70112339F08C2F0E94940D8D2F0E9431
:1017C000390A6EC08D2F0E94400A8C2F0E94B50DE1
:1017D00067C0D23F21F128F4D03F41F0D13FC1F0A2
:1017E00043C0D33F19F1D43F79F03EC0112341F0FB
:1017F000053008F051C08C2F8F710E94DA0D4CC05B
:10180000063008F049C0F7CF80910D0382FF18C061
:10181000112339F08C2F8F710E94940D3DC011233C
:10182000C9F38C2F8F710E94B50D36C0112329F09A
:101830008C2F8F710E947F0D2FC00E947A0D2CC0BB
:10184000112349F0CF718C2F0E94940D63E08C2FEF
:101850000E94B61221C081E00E94D1120230E0F055
:1018600082E00E94D11218C0112331F0002391F2BE
:101870008D2F0E94020910C0002399F2D93349F438
:101880001FEF27EE33E0115020403040E1F700C059
:1018900000008D2F0E94B10988EF8C0D843020F458
:1018A0000E94B6230E947008DD20C9F00E94241215
:1018B00080FD15C0F70112820E941E120E94940D35
:1018C000C7010E94900C0E941E12DF91CF911F91C0
:1018D0000F91FF90EF90DF90CF900C94B50DDF91BA
:1018E000CF911F910F91FF90EF90DF90CF900895CF
:1018F0000F931F93CF93DF93EC01688179818A81E5
:101900000E94D60E8C010E94310E0E94220DB80159
:10191000CE010E94470ADF91CF911F910F91089548
:10192000CF93DF93EC01988189812B813C81232B1C
:1019300031F08F3F31F481E09F3F19F403C081E023
:1019400001C080E080FD1DC0CE010E94BE07811154
:1019500010C00E9428128823A1F08A81882389F070
:1019600080910D0382FD0DC082E0DF91CF910C9438
:10197000D112CE010E94780CCE01DF91CF910C9450
:101980009F07DF91CF91089580E090E00E94252489
:1019900080E090E00E943B240E944F120E9471124E
:1019A0000E94D51B0C94221A809102019091030190
:1019B0000E941F250C94C40C0E943F120C94D40C5E
:1019C00092959F70963079F010F4925001C09A5021
:1019D000923068F4803F69F018F4883E40F409C002
:1019E000843F29F406C0883E20F0813F11F080E05A
:1019F000089581E00895FC01808191810E94CB0EC1
:101A00000E94E00C0895CF93DF9300D000D01F9286
:101A1000CDB7DEB70F900F900F900F900F90DF9122
:101A2000CF910895CF93DF9300D000D000D0CDB7F1
:101A3000DEB726960FB6F894DEBF0FBECDBFDF919E
:101A4000CF910895089508950C94230D0C94240DBE
:101A50000E94260D60932F02709330028093310212
:101A6000909332020C94C40C0C94280D0F931F9386
:101A700000912F02109130022091310230913202F8
:101A8000602B712B822B932B1F910F910C94280D9F
:101A90000F931F9300912F02109130022091310279
:101AA0003091320260237123822393231F910F917F
:101AB0000C94280D0F931F9300912F021091300268
:101AC00020913102309132026027712782279327BB
:101AD0001F910F910C94280D0C94230D0E946C0DF6
:101AE00060932B0270932C0280932D0290932E0210
:101AF0000C94C40C60E070E0CB010C946E0D0F935D
:101B00001F9341E050E060E070E08A019B0104C057
:101B1000000F111F221F331F8A95D2F7C901B80188
:101B20001F910F910C946E0D0F931F9341E050E0A5
:101B300060E070E004C0440F551F661F771F8A9550
:101B4000D2F780912B0290912C02A0912D02B0919E
:101B50002E028A019B01082B192B2A2B3B2BC90132
:101B6000B8011F910F910C946E0D0F931F9341E0DC
:101B700050E060E070E004C0440F551F661F771FFF
:101B80008A95D2F7409550956095709580912B027B
:101B900090912C02A0912D02B0912E028A019B01FE
:101BA000082319232A233B23C901B8011F910F9150
:101BB0000C946E0D0F931F9341E050E060E070E0D5
:101BC00004C0440F551F661F771F8A95D2F7809176
:101BD0002B0290912C02A0912D02B0912E028A012D
:101BE0009B01082719272A273B27C901B8011F9104
:101BF0000F910C946E0D0F931F9300912B02109177
:101C00002C0220912D0230912E02602B712B822B01
:101C1000932B1F910F910C946E0D0F931F930091B6
:101C20002B0210912C0220912D0230912E02602364
:101C30007123822393231F910F910C946E0D0F93A8
:101C40001F9300912B0210912C0220912D023091B4
:101C50002E0260277127822793271F910F910C94E2
:101C60006E0D08952EE0929F800D1124E82FE695C9
:101C7000E695E695877051E001C0550F8A95EAF721
:101C800085E0E89FF0011124E250FE4F20E030E0B3
:101C900070E04081CB01022E02C0969587950A9490
:101CA000E2F78170819584278523842781932F5FB4
:101CB0003F4F2530310569F708952EE0929F800D42
:101CC0001124682F669566956695982F977085E024
:101CD000689FB001112440E050E080E0FB01E40F78
:101CE000F51FE250FE4F208130E0092E02C03695EC
:101CF00027950A94E2F721703327042E01C0220FA2
:101D00000A94EAF7822B4F5F5F4F4530510531F758
:101D10000895BF92CF92DF92EF92FF920F931F939D
:101D2000CF93DF938C01C0902B02D0902C02E090D7
:101D30002D02F0902E0280912F0290913002A091FE
:101D40003102B0913202C82AD92AEA2AFB2ACFE10D
:101D5000D0E0D701C6010C2E04C0B695A795979583
:101D600087950A94D2F780FD04C0219790F7B12C93
:101D700007C0BC2EB8018C2F0E94EC150197A9F367
:101D80008B2DDF91CF911F910F91FF90EF90DF90FE
:101D9000CF90BF900895CF93DF93EC010E94890EFE
:101DA000BE010E94EC15DF91CF9108951F93CF9350
:101DB000DF93EB019091FD01992321F0CB010E946B
:101DC000CB0E13C0882349F0CB010E94890E182F37
:101DD000682FCE010E94320E04C0CB010E945D0E1E
:101DE000182FBE01812F0E94EC15DF91CF911F911A
:101DF00008951F93CF93DF93C091330216E0809133
:101E00003402C81799F0D0E01C9FF0011D9FF00D1F
:101E10001124EB5CFD4F408151816281738184818B
:101E200095810E94120D2196C770E9CFDF91CF9165
:101E30001F9108954091650250916602609167027A
:101E4000709168028091690290916A020C94120D5F
:101E5000EF92FF920F931F93CF93DF9380916A02CB
:101E600082958F7009F065C080916702882309F41C
:101E700060C080913302F0903402109165020091AD
:101E80006602609168027091690291E01F3F09F05B
:101E900090E0C0910001D0910101292F96E0E92E38
:101EA0008F1509F446C06115710521F00F3F21F02F
:101EB00030E003C031E001C0322F90E030FD36C089
:101EC000E89EF001E99EF00D1124DF01AB5CBD4FEF
:101ED00011963C911197301329C03C91311326C0C3
:101EE00012963C911297311121C013964D915C913D
:101EF0001497461B570B4C175D07C0F480916A027C
:101F00008F70806180936A02E65CFD4F80818F70E4
:101F10008061808385E692E00E94900CDF91CF91F2
:101F20001F910F91FF90EF900C94F90E019687701E
:101F3000B7CFDF91CF911F910F91FF90EF90089550
:101F40009F92AF92BF92CF92DF92EF92FF920F9348
:101F50001F93CF93DF93CDB7DEB761970FB6F89499
:101F6000DEBF0FBECDBF8C0185E0F801DE011D96FE
:101F700001900D928A95E1F7D8011296EC9090911C
:101F80006502E09166022091680230916902211594
:101F9000310531F0EF3F31F481E09F3F19F403C088
:101FA00081E001C080E0B82FB1709B2E80FD47C159
:101FB000D8014C9111965C9111971396AD90BC90FD
:101FC000149785E6C82E82E0D82EF0906702B501FE
:101FD000621B730B2091000130910101FF2009F475
:101FE000D9C080916A026217730708F095C0282F44
:101FF000207F09F052C05E1313C0491311C0FE2C9C
:10200000E1100EC08F70806180936A020E941A0FE7
:10201000C6010E94900C80916A02F80185834DC12F
:10202000AB2831F05F3F31F481E04F3F19F403C03A
:1020300081E001C080E080FD03C081E08E2502C008
:1020400080E090E0F82FF170FF2E80FF1CC080919F
:1020500033022091340236E0821709F40BC190E07C
:10206000389FF001399FF00D1124EB5CFD4F618129
:10207000561306C06081461303C06281E61203C096
:1020800001968770E9CFFE2CEE2009F416C18091ED
:102090006A02816080936A0254C05E1306C04913CD
:1020A00004C0E11002C0F80199C0C8010E94FB0CF5
:1020B000882361F1EE2051F120916A02822F8295EE
:1020C0008F7090E0029774F08091650290916602A3
:1020D00098878F831986BB86AA862C87CE010796A0
:1020E0000E94900C86E0F801A5E6B2E001900D9206
:1020F0008A95E1F70E94280F0E941A0F0AC05E1706
:1021000011F1C8010E94FB0C81112CC0C8010E9472
:10211000900CFF24F394D1C0282F207F81F77A2DD3
:10212000B98AA88A6E2D89890E94030D85E692E0FE
:102130000E94900C86E0D6011D928A95E9F70E94D4
:102140001A0FF12CBAC04913DCCFE110DACFF80135
:102150008583C8010E94900C86E0D6011D928A9565
:10216000E9F7ABC0EE2091F220916A02822F8295AE
:102170008F7090E002970CF4B5CF8091650290913A
:1021800066029A8389831B82BD82AC822E83CE0134
:102190000196A6CF6217730708F044C0FE2CEE200C
:1021A00009F4B4CF5E1330C049132EC020916A02E7
:1021B00020FD21C0822F82958F70482F50E041155D
:1021C0005105C9F0F80125834F30510541F08F5F6B
:1021D000982F9295907F822F8F70892B8583C801CD
:1021E0000E94900C86E0F801A5E6B2E001900D9205
:1021F0008A95E1F73CC086E0F801A5E6B2E00190DF
:102200000D928A95E1F759C0C8010E94FB0C81111B
:1022100069CF80916A02816080936A02C8010E943E
:10222000900C4BC07A2DB98AA88A6E2D89890E949C
:10223000030D86E0D6011D928A95E9F718C0EE20BD
:1022400009F464CFC8010E94FB0CF82E882309F41E
:102250005DCF86E0F801A5E6B2E001900D928A9587
:10226000E1F785E692E00E94FC080E94280F0E9498
:102270001A0F23C04D875E878D859E850E94CB0EE9
:10228000292F22952F70223028F49F7039F0811168
:1022900005C00BC0243028F49F7049F4805E88305C
:1022A00020F0C8010E94900C9F2CF92C06C0D80188
:1022B00015969C91907F91F7F8CF8F2D61960FB670
:1022C000F894DEBF0FBECDBFDF91CF911F910F916C
:1022D000FF90EF90DF90CF90BF90AF909F900895C8
:1022E0001F93CF93DF93CDB7DEB72C970FB6F8943B
:1022F000DEBF0FBECDBF4F83588769877A878B8734
:102300009C87CE0107960E94A00F8823D1F09F8161
:1023100088852A853B85232B31F08F3F31F481E07E
:102320009F3F19F403C081E001C080E080FD47C0F9
:102330004F81588569857A858B859C850E94120D11
:102340003EC086E0FE013796DE01119601900D92A7
:102350008A95E1F7FF81E8856A857B8561157105BE
:1023600031F0EF3F31F481E0FF3F19F403C081E029
:1023700001C080E080FD23C02091340230E0C9011B
:102380000196877099274091330250E08417950792
:10239000F1F1F983EA837D836C8396E0929FD0010B
:1023A000939FB00D1124AB5CBD4FFE01319601909F
:1023B0000D929A95E1F7809334020E94F90E16E08F
:1023C0008091330290913402891771F1189FC001F6
:1023D00011248B5C9D4F0E94A00F882329F1E0916E
:1023E00033021E9FF0011124EB5CFD4F40815181AF
:1023F00062817381848195810E94120D80913302E4
:1024000090E001968770992780933302D9CF0E947C
:10241000DC0C1092340210923302E5E6F2E086E022
:10242000DF011D928A95E9F72C960FB6F894DEBF6E
:102430000FBECDBFDF91CF911F91089580918B0288
:10244000859585958595089580918B02877008956F
:1024500090918B02977081E009F480E0089580915B
:10246000AE0208959091AE02892B8093AE0208953A
:1024700080959091AE0289238093AE0208951092C8
:10248000AE0208959091AD02892B8093AD0208951C
:1024900080959091AD0289238093AD0208951092AA
:1024A000AD02089580918C02089508950C94551200
:1024B0000C94561290910D0392FD08C090918C02DD
:1024C000981721F080938C020C94581208958091F3
:1024D0008C02882329F010928C0280E00C94581210
:1024E0000895CF93DF93E0910201F0910301809171
:1024F000AE028083E0910201F0910301908180910E
:10250000AD02892B808380918C02882381F0E09139
:102510000201F09103019081892B80838091020157
:10252000909103010E94512481110E946712C09171
:102530000201D091030140E250E06BE672E0CE016F
:102540000E94622E892B69F080E2FE01ABE6B2E0C8
:1025500001900D928A95E1F7CE01DF91CF910C9415
:10256000C223DF91CF9108950C94551290910D03E1
:1025700092FD10C098E0899F90011124262B209392
:102580008B020E94940D80918B028595859585958F
:102590000C94B4120C94940D10928B0280E00C9465
:1025A000B41220918B028095822380938B02982F06
:1025B000977099F430E0482F082E000C550B241723
:1025C000350759F090910D0392FD07C085958595CB
:1025D00085950E94B50D0C94CC120895CF939091DF
:1025E0000D0392FB222720F92817F9F0C82F892F15
:1025F000C0FB82F980930D0380910C0390910D0331
:102600000E94501382E00E94D1128091C10280FF8B
:102610000CC01F92CF9383EA92E09F938F930E9406
:102620004F070F900F900F900F90CF9108958091CA
:102630000D0382FB882780F991E089270C94EE1224
:1026400081E00C94EE1280E00C94EE126FEF7FEFBD
:1026500080E090E00C949B2E80E090E00E94772E2A
:1026600021E0893E9E4F09F020E0822F089582E00C
:1026700090E00C946F2E83E090E00C946F2ECF933B
:1026800084E090E00E946F2EC82F82E290E00E94CA
:102690006F2E2C2F30E0A901582BCA01CF9108953D
:1026A000CF93C92F682F84E090E00E947D2E6C2F7D
:1026B00082E290E0CF910C947D2EAB01BC018FE0C3
:1026C00090E00C948F2EAB01BC0183E190E00C9460
:1026D0008F2E60E070E0CB010C94631360E070E03B
:1026E000CB010E945D130C94691369EE7EEF80E0CC
:1026F00090E00E949B2E60E082E090E00E947D2EA0
:1027000060E083E090E00E947D2E10922F021092F4
:102710003002109231021092320260E084E090E0C8
:102720000E947D2E60E082E290E00E947D2E60E0BB
:1027300085E090E00E947D2E60E086E090E00E94BF
:102740007D2E6FEF87E090E00E947D2E40E050E00C
:10275000BA0188E090E00E948F2E60E08DE090E06A
:102760000E947D2E40E050E0BA0188E190E00E9496
:102770008F2E60E087E190E00E947D2E40E050E0E7
:10278000BA018CE190E00E948F2E60E070E080E260
:1027900090E00E949B2E40E050E0BA0188E190E07A
:1027A0000E948F2E0C946E130C947513682F8EE07C
:1027B00090E00C947D2E0E94D9256093BD02709309
:1027C000BE028093BF029093C0026093B9027093DF
:1027D000BA028093BB029093BC02089585B78068CB
:1027E00085BF85B7806885BF089581E008950C9402
:1027F000F51308950C94F9130C94F9130C94FC132D
:102800000C94F9130C9400140C94F9130E94EE1319
:1028100086E298E20E94AC230E9404140C940214F5
:102820000E94FA130C94F9130E94E0160E946F089C
:102830000C94271E0E94C4250E941A180E9414148A
:102840000E94F41B0C94FE135F926F927F928F9202
:102850009F92AF92BF92CF92DF92EF92FF920F932F
:102860001F93CF93DF93CDB7DEB72A970FB6F894B7
:10287000DEBF0FBECDBF0E942F18C82E81110E944F
:10288000DB133FEA832E32E0932E00E010E0502E5F
:10289000802F0E9404175C01F401619071904F0138
:1028A0006826792661147104B1F40F5F1F4F05305B
:1028B000110569F78FEF89838A831B820E94CD25DA
:1028C0008160782F9D838C8349815A816B818D81B2
:1028D0000E94B2083AC08091C10281FD0E940D178A
:1028E000D12CEE24E394F12CC3018E219F21892B5E
:1028F00029F10E94F7138823A9F0DE825F82AE20BF
:10290000BF2081E0AB2809F480E088870E94CD25B4
:102910008160782F9A8789874E815F8168858A8553
:102920000E94B208000F111FF801E155FD4F808190
:102930009181E826F926F182E08207C0D394EE0C5B
:10294000FF1CFEE0DF12D0CFB0CF81E0C11001C08C
:1029500080E02A960FB6F894DEBF0FBECDBFDF91A0
:10296000CF911F910F91FF90EF90DF90CF90BF908C
:10297000AF909F908F907F906F905F9008950E948E
:1029800024140E94261E0E94C21A0C948008CF9321
:10299000DF930E94F115EC01811521E5920708F003
:1029A00045C0811530E5930708F094C0883E910535
:1029B00028F5803E910508F0F8C0883A910570F43A
:1029C000853A910508F07CC08130910509F475C005
:1029D00008F4E8C0049708F0E8C0E4C08F3B910514
:1029E00008F0E0C0C85AD0E0CC0FDD1FC65BDE4F58
:1029F0000990D881C02DCE019464D8C0811540E2E1
:102A0000940758F4811551E0950708F0CEC08D3E2B
:102A1000910508F4C7C09065C9C0C11580E4D80706
:102A200008F4C0C0DF70CE01906AC0C0811525E5F2
:102A30009207A8F4811534E5930708F095C0811535
:102A400043E5940708F07BC0811552E5950708F02F
:102A500061C0D82FCC27CE01816F906AA7C0C11565
:102A600089E5D807A0F4C11528E5D20708F082C08F
:102A7000C11536E5D30708F095C08C2F0E94851646
:102A80008F7190E0D82FCC27CE0190628FC0C115F6
:102A90004AE5D40708F474C0CE01905681159042DF
:102AA00008F080C08D2F8F710E948516DD27D062BF
:102AB0008F71AE01582BCA0179C081E090E076C0D9
:102AC000C55AD0E0C858DE4F8881C82FD0E0CE016B
:102AD00090646CC074E0969587957A95E1F7282FFD
:102AE00023703C2F337081E090E002C0880F991F63
:102AF0003A95E2F79C68AC01522B9A019C2F9F708B
:102B00009695969550E2959FE0011124C9018C2B72
:102B10009D2B4CC08370992721E030E002C0220F2A
:102B2000331F8A95E2F79C2F9695969580E2989FA1
:102B3000E0011124C22BD32BCE019C6837C08370D7
:102B4000992721E030E002C0220F331F8A95E2F777
:102B50009C2F9695969540E2949FE0011124C22BFC
:102B6000D32BCE019A6822C0D82FCC27CE01846FF8
:102B7000906A1CC0DC2FCC27CE01806F906A16C0F3
:102B80008C2F8F700E94851694E0D695C7959A95E4
:102B9000E1F7CF70D0E0DC2FCC27D0699E01282B45
:102BA000C90104C080E090E001C0CE01DF91CF9167
:102BB000089526E4829FC0011124FC012EE0729F3B
:102BC000E00DF11D1124E60FF11DEE0FFF1FEA5A73
:102BD000FE4F8591949108950E94D9150E94C714C3
:102BE00008958238910569F1B0F48133910509F4B3
:102BF0006DC048F48932910509F463C08A329105A9
:102C000009F469C008958533910509F455C08933E5
:102C10009105B9F00895833E910569F138F4803E3D
:102C20009105B1F0823E910509F10895863E910526
:102C3000A9F1873E9105B9F1843E910509F064C080
:102C400023C020910C0320FD4FC021FD4DC00895ED
:102C500080910C0380FD44C080910D0380FF44C02F
:102C600080910C0384FD42C083EE4DC080910C0323
:102C700082FF38C0F5CF80910C0382FD33C0809174
:102C80000D0380FD31C0ECCF80910D0381FF32C078
:102C900080910C0384FD2AC087EE35C080910C031F
:102CA00083FF26C0F5CF80910C0383FD21C0809166
:102CB0000D0381FD1FC0ECCF80910C0385FD1CC06E
:102CC0001DC080910C0385FD19C016C080910C03B6
:102CD00086FD16C017C080910C0386FD13C010C07E
:102CE00089E311C082EE0FC080EE0DC080E00BC002
:102CF00086EE09C084EE07C089E205C085E303C003
:102D00008AE201C081E390E0089590910C0392FF64
:102D10000DC0282F2871283019F4877F846006C0E1
:102D2000282F2471243011F48B7F886093FF0DC00D
:102D3000282F2871283119F4877E846106C0282F36
:102D40002471243111F48B7E886120910D0320FFC2
:102D50000DC0382F3871383019F4877F816006C074
:102D6000382F3171313011F48E7F886021FF0DC012
:102D7000282F2871283119F4877E816106C0282FF9
:102D80002171213111F48E7E886194FD877E089532
:102D90000C9426130E942F188FE39CE90197F1F7FA
:102DA00000C000000E942F1880E00E94041780FFDE
:102DB00004C00E94C8160C941A2608950C94CA16D2
:102DC0000E942C13811102C00E94D4130E94371359
:102DD0008093C1020E943F1390930D0380930C03D4
:102DE0000E94DE160E943B13682F70E080E090E0A6
:102DF0000E94340D60912B0270912C0280912D0263
:102E000090912E020C946C0DE82FF0E0EE0FFF1F56
:102E1000E85EFC4F808191810895CF92DF92EF921E
:102E2000FF920F931F93CF93DF9388EC92E00E9461
:102E3000B60688E1E82E83E0F82EC0E0D0E093ECFF
:102E4000C92E92E0D92E0AEB12E0DF93CF93DF92E6
:102E5000CF920E944F0780EC92E00E94B606F701E5
:102E6000819191917F010E9455089F938F931F93A9
:102E70000F930E944F0788EB92E00E94B6062196BE
:102E80008DB79EB708960FB6F8949EBF0FBE8DBF44
:102E9000C530D105D1F6DF91CF911F910F91FF90F1
:102EA000EF90DF90CF90089580EA8A95F1F708952A
:102EB00000C008950C94541708950C945C170C945A
:102EC0005D170C945C170C946117F894E82FE29549
:102ED000EF70F0E031A1282F2F7081E090E001C069
:102EE000880F2A95EAF7982F9095932391A392A1A2
:102EF000892B82A3789408950F931F93CF93DF9328
:102F0000CBE7D1E089918F3F11F00E94651781E0F6
:102F1000C938D807B9F7C9E8D1E00EE811E08991BE
:102F20008F3F11F00E9465170C171D07C1F7DF9145
:102F3000CF911F910F910895AF92BF92DF92EF92C0
:102F4000FF920F931F93CF93DF93C62FD0E0C55806
:102F5000DE4F28812F3F09F463C08A01F62EE92E47
:102F6000D82EF894E22FE295EF70F0E091A1822F35
:102F70008F7021E030E001C0220F8A95EAF7892F97
:102F8000822B81A382A12095282322A378940E94DA
:102F9000581789E8A82E81E0B82EED2DFE2D9F014F
:102FA000265F3F4FE12CA80140955095D5016D91CA
:102FB0005D016F3FC9F0862F82958F7090E0DC0134
:102FC00090968C9190E06F7002C0959587956A9568
:102FD000E2F780FD09C080819181802B912B918344
:102FE0008083EE24E39406C080819181842395231D
:102FF000918380833296E217F307C1F688818F3F71
:1030000011F00E9465176E2D8F2DDF91CF911F91CA
:103010000F91FF90EF90DF90BF90AF900C945A17F4
:10302000DF91CF911F910F91FF90EF90DF90BF90B4
:10303000AF9008950E947C178AE0E8E1F3E0DF0199
:10304000982F1D929A95E9F7EEE0F3E0DF011D92CB
:103050008A95E9F785E00E9484180C94AA07CF921C
:10306000DF92FF920F931F93CF93DF93CDB7DEB71D
:103070002A970FB6F894DEBF0FBECDBF8E010F5F4B
:103080001F4F8AE0F80111928A95E9F7F12CCC24C0
:10309000C394D12CA6016F2DC8010E949C17F394F4
:1030A000CC0CDD1CFEE0FF12F5CF4AE050E0B80189
:1030B0008EE093E00E94622EFF24F394009709F4BF
:1030C000F12C892B41F08AE0F801AEE0B3E00190E9
:1030D0000D928A95E1F72F2D45E068E173E08EE0CF
:1030E00093E00E9485180E94AC078F2D2A960FB698
:1030F000F894DEBF0FBECDBFDF91CF911F910F912E
:10310000FF90DF90CF9008950895FF920F931F9343
:10311000CF93DF93F82E092F162FD72FC42F2223FA
:1031200049F081E08093C4020E94CD259093C302B0
:103130008093C2028091C4028823D9F08091C20298
:103140009091C3020E94E525059798F0EF2DF02F8E
:10315000A12FBD2F80E090E04C2F50E08417950701
:1031600034F4219131912D933D930196F7CF109234
:10317000C402DF91CF911F910F91FF9008950E949B
:10318000A2280E941A140C94AE280E94B2280E9411
:10319000BF140C94D0280E946B250E9489280E949D
:1031A00006140E94BF180E94C5180E941014FBCF7D
:1031B0008091CB0280FF06C06091090170E0660F2C
:1031C000771F26C081FF04C06091090184E005C01B
:1031D00082FF07C06091090188E0689FB001112457
:1031E00017C09091CA029923D1F0609108019617F7
:1031F00088F72091090188E0289F90011124929F6F
:10320000A001939F500D112470E0CA010E940C2E62
:103210006038710540F46115710519F406C068E065
:1032200070E0862F08958FE7089581E008958091DA
:10323000CB0280FF08C06091050170E0759567952D
:103240007595679521C081FF06C06091050170E00A
:103250007595679519C082FF04C06091050170E003
:1032600010C09091C902992399F0609104019617BA
:10327000A0F780910501899FC001112470E00E9490
:103280000C2E6038710540F46115710519F406C003
:1032900061E070E0862F08958FE7089581E008953A
:1032A0008D3E21F40E94D818819504C08E3E29F4E9
:1032B0000E94D8188093CF0208958F3E21F40E9477
:1032C000D818819504C0803F29F40E94D8188093B3
:1032D000CE020895893F19F40E94171905C08A3F4C
:1032E00031F40E94171981958093D00208958B3F85
:1032F00021F40E941719819504C08C3F29F40E9483
:1033000017198093D10208959FE0980F983078F4B0
:1033100021E030E0A90102C0440F551F9A95E2F761
:10332000CA019091CD02892B8093CD0208958D3FE3
:1033300021F48091CB0281600BC08E3F21F48091FB
:10334000CB02826005C08F3F29F48091CB0284605C
:103350008093CB0208958D3E39F49091CF0297FF70
:1033600035C01092CF0259C08E3E29F49091CF0201
:103370001916BCF32BC09091CE028F3E29F497FF13
:1033800025C01092CE0249C0803F19F41916CCF323
:103390001DC09091D002893F29F41916BCF41092F7
:1033A000D0023BC08A3F19F497FF10C0F8CF8B3F83
:1033B00039F49091D10297FF09C01092D1022DC02B
:1033C0008C3F21F49091D1021916BCF39FE0980F25
:1033D000983080F421E030E0A90102C0440F551F6D
:1033E0009A95E2F7CA0180959091CD028923809346
:1033F000CD0213C08D3F21F48091CB028E7F0BC094
:103400008E3F21F48091CB028D7F05C08F3F29F440
:103410008091CB028B7F8093CB028091CE02811171
:1034200006C08091CF02811102C01092CA02809121
:10343000D002811106C08091D102811102C0109288
:10344000C90208958091C10283FF7EC086E093E0A7
:103450000E94B6068091CD021F928F9381E093E087
:103460009F938F930E944F078FEF92E00E94B606C2
:103470008091CE02282F082E000C330B3F938F93A0
:103480008CEF92E09F938F930E944F078AEF92E018
:103490000E94B6068091CF02282F082E000C330B15
:1034A0003F938F9387EF92E09F938F930E944F07F4
:1034B00085EF92E00E94B6068091D002282F082E58
:1034C000000C330B3F938F9382EF92E09F938F9387
:1034D0000E944F0780EF92E00E94B6068091D102D1
:1034E000282F082E000C330B3F938F938DEE92E024
:1034F0009F938F930E944F078AEE92E00E94B60638
:103500008091CA021F928F9387EE92E09F938F93D0
:103510000E944F0785EE92E00E94B6068091CB0292
:103520001F928F9382EE92E09F938F930E944F079A
:103530008FED92E00E94B6068DB79EB74C960FB6FF
:10354000F8949EBF0FBE8DBF0E94CD252091CE0264
:10355000211104C02091CF02222321F09093C802B0
:103560008093C7022091D002211104C02091D10282
:10357000222321F09093C6028093C5028CEC92E046
:103580000C941724EF92FF920F931F93CF93DF9326
:1035900000D000D000D0CDB7DEB786E0ECECF2E092
:1035A000DE01119601900D928A95E1F7E090CE022E
:1035B000F090CF020091D0021091D1021092CE0271
:1035C0001092CF021092D0021092D102E11003C0EB
:1035D000FF2009F45DC08091C7029091C8020E944B
:1035E000E525AC019091CA02992339F020910A0196
:1035F00030E02417350758F04BC020910B018AE0CA
:10360000289F900111242417350718F041C09F3FCF
:1036100019F09F5F9093CA02EE2061F00E94D818C3
:103620001E1414F09FEF01C091E0989F902D11247B
:103630009093CE02FF2061F00E94D8181F1414F05E
:103640009FEF01C091E0989F902D11249093CF029D
:103650003091CE023323E1F02091CF022223C1F03A
:1036600045EB3403C0011124992319F09093CE0245
:1036700003C081E08093CE0235EB2303C001112407
:10368000992319F09093CF0203C081E08093CF0279
:10369000011103C0112309F45DC08091C50290910E
:1036A000C6020E94E525AC019091C902992339F028
:1036B0002091060130E02417350758F04BC02091C7
:1036C00007018AE0289F900111242417350718F07C
:1036D00041C09F3F19F09F5F9093C902002361F0A2
:1036E0000E941719101614F09FEF01C091E0989FE7
:1036F000902D11249093D002112361F00E9417198C
:10370000111614F09FEF01C091E0989F902D1124A5
:103710009093D1023091D0023323E1F02091D10275
:103720002223C1F045EB3403C0011124992319F081
:103730009093D00203C081E08093D00235EB230345
:10374000C0011124992319F09093D10203C081E0A4
:103750008093D1028091CE0281110BC08091CF0263
:10376000811107C08091D002811103C08091D102E4
:1037700081110E94221AEB82FC820D831E8386E057
:10378000FE013196ACECB2E001900D928A95E1F722
:1037900026960FB6F894DEBF0FBECDBFDF91CF9156
:1037A0001F910F91FF90EF900895ECECF2E086E00E
:1037B000DF011D928A95E9F71092CA021092C902A0
:1037C0001092CB02089586E090E00C946F2E682F43
:1037D00086E090E00C947D2E8091220384708961B4
:1037E000809322030C94E71B0E942C13811104C0C8
:1037F0000E94D4130E94EC1B0E94E31B80932203BF
:10380000282F26952695269530E02430310524F082
:1038100087708861809322038091220380FF04C017
:1038200086958695869501C080E00C94711D209147
:103830002203822F869586958695482F50E0433047
:10384000510554F48F5F982F990F990F990F822F7C
:103850008770892B8093220380912203816080935B
:1038600022030E94E71B8091C10280FF11C080915A
:1038700022038695869586951F928F9380E993E023
:103880009F938F930E944F070F900F900F900F9070
:10389000809122038695869586950C94711D809162
:1038A0002203982F969596959695A1F0915E990F83
:1038B000990F990F8770892B80932203887F91E05D
:1038C00009F490E08091220390FB80F98093220319
:1038D0000E94E71B8091C10280FF11C080912203EA
:1038E0008695869586951F928F9388E793E09F93A0
:1038F0008F930E944F070F900F900F900F90809121
:1039000022038695869586950C94711D80912203DD
:1039100080FD1FC0816080932203813019F489E00B
:1039200080932203809122030E94E71B8091C102B1
:1039300080FF08C080E593E09F938F930E944F071C
:103940000F900F90809122038695869586950C9412
:10395000711D08958091220380FF14C08E7F809393
:1039600022030E94E71B8091C10280FF08C08DE303
:1039700093E09F938F930E944F070F900F9080E0EA
:103980000C94711D0895CF93C0912203C170809152
:10399000C10280FF0CC01F92CF9382E693E09F93F9
:1039A0008F930E944F070F900F900F900F90CC2392
:1039B00019F0CF910C94AA1CCF910C94861C909175
:1039C0002203892F8695869586958F5F8F719770D4
:1039D000843038F4880F880F880F892B8093220356
:1039E00002C09093220380912203887F91E009F422
:1039F00090E08091220390FB80F9809322030E9443
:103A0000E71B8091C10280FF11C08091220386953F
:103A1000869586951F928F9389E293E09F938F936B
:103A20000E944F070F900F900F900F9080912203EC
:103A30008695869586950C94711D843008F083E0F8
:103A4000909122039770282F220F220F220F922B82
:103A500090932203987F21E009F420E090912203C3
:103A600020FB90F9909322030C94711D0E941D1D60
:103A7000809122030C94E71B9C01FB018281882327
:103A800049F12E3BFCE53F07C9F040F42C3BECE547
:103A90003E0769F02D3B3C4561F00895203C9CE5D4
:103AA000390791F070F0213C3C4589F0089583E09E
:103AB00001C080E00E94361D80E008950E944F1CE6
:103AC000FBCF0E94171CF8CF0E94C31CF5CF0E94A9
:103AD000DF1CF2CF81E00895279A2F9808952F9840
:103AE00008958F929F92AF92BF92CF92DF92EF9202
:103AF000FF920F931F93CF93DF93C82F843050F41E
:103B0000811109C080918000877F809380000E948E
:103B10006F1D06C0C3E080918000886080938000A4
:103B2000A0918600B09187002C2F30E00E94482E93
:103B300023E030E040E050E00E94202E0027122FCA
:103B4000232F342F012F122F232F3327809186000C
:103B5000909187006CE070E00E94F82D601771076B
:103B600030F0C80169E070E00E94F82D5EC08091DD
:103B7000860090918700E0908600F0908700E091A9
:103B80008600F0918700C6E0D0E0BE010E94F82DCB
:103B9000060F171F211D311D4801590185E0880CB2
:103BA000991CAA1CBB1C8A95D1F7C701BE010E94B3
:103BB000F82D6F01E12CF12CA7019601260F371F7C
:103BC000411D511DC501B4010E94202E69017A01D9
:103BD000E0918600F0918700CA01B9010E94DC2DB6
:103BE0009B01AC01DF010E94572E9B01AC01C70174
:103BF000B6010E94DC2DDC01CB012FE0B695A79524
:103C0000979587952A95D1F70091860010918700A6
:103C100020E030E0081719072A073B0728F46091D5
:103C2000860070918700CB01BC0170938D0060937A
:103C30008C00DF91CF911F910F91FF90EF90DF905B
:103C4000CF90BF90AF909F908F90089508950E945D
:103C50006C1D8AE08093800089E1809381008FEF62
:103C60009FEF90938700809386000C94F41BCF9372
:103C7000DF93EC01FB018281882309F43CC1C4304D
:103C8000FDE5DF0760F4CB3F9CE5D90788F49E0192
:103C900022503C452431310508F02EC109C0C236FE
:103CA000EDE5DE0729F0C63AFDE5DF0709F024C19E
:103CB0000E943F1390930D0380930C03C1318CE558
:103CC000D80709F4C6C008F042C0C930ECE5DE07E9
:103CD00009F49BC000F5C5308CE5D80709F485C010
:103CE00078F4C330ECE5DE0709F478C008F07AC058
:103CF000C230DC4509F0F5C080910C038160EFC053
:103D0000C7309CE5D90709F478C008F07AC08091E3
:103D10000C038061E4C0CD30FCE5DF0709F487C007
:103D200058F4CB309CE5D90709F479C008F07BC082
:103D300080910C0388606FC0CF30FCE5DF0709F489
:103D400080C008F082C080910C03877FC8C0CE3F3E
:103D50009CE5D90709F471C000F5C531FCE5DF0722
:103D600009F485C068F4C3319CE5D90709F475C02E
:103D700008F095C00E94DC0C80910C038F77AFC0D7
:103D8000CC3FFCE5DF07A9F108F054C0CB3FDC4590
:103D900009F0A7C080910D0340C0C230EDE5DE07F9
:103DA00009F489C058F4C1158DE5D80709F45AC043
:103DB00008F069C080910D0382602FC0C236EDE526
:103DC000DE0709F47CC0C63AFDE5DF0709F481C0CF
:103DD000C330DD4509F085C080E06EC080910C03E2
:103DE00082607DC080910C0316C080910C038860B6
:103DF00076C080910D0382604FC080910C03806279
:103E00006EC080910C0380646AC00E94DC0C8091BB
:103E10000C03806864C0846062C081603DC0809192
:103E20000C038E7F5CC080910C038D7F58C0809105
:103E30000C0316C080910D0318C080910D038D7F77
:103E40002BC080910C038F7E4AC080910C038F7D24
:103E500046C080910C038F7B42C080910C03877F0A
:103E60008B7F3DC080910D038D7F8E7F15C080912B
:103E70000C0382FB222720F991E0922790FB82F924
:103E800090FB83F92CC080910D03982F9095917031
:103E90008E7F892B90FB81F980930D0322C00E94B5
:103EA000DC0C80910C0387FB222720F991E09227FC
:103EB00090FB87F914C081E00E94D61312C0809154
:103EC0000C0384FB222720F991E0922790FB84F9D0
:103ED00006C080910C03982F909590FB80F98093F9
:103EE0000C0380910C0390910D030E9450130E94CB
:103EF000DC0C80E001C081E0DF91CF9108958091DA
:103F000004011F928F93809105011F928F938091DE
:103F100008011F928F93809109011F928F938091C6
:103F20000A011F928F9380910B011F928F9388EA51
:103F300093E09F938F930E944F078DB79EB70E9685
:103F40000FB6F8949EBF0FBE8DBF0895883220F53E
:103F50008E3108F068C08B3091F1C0F4873009F0E1
:103F6000BEC081E080930B0184E180930A018AE066
:103F7000809309018EE18093080188E08093050118
:103F800088E2809304018AE095E0C6C0833109F499
:103F900043C0843169F1A3C08F3409F49EC028F472
:103FA000893231F1883359F09AC0813531F008F403
:103FB000D4C0823509F4A7C092C08FEFA5C08CE2AF
:103FC00095E00E94B6060E947F1F1F9281E08F93AA
:103FD0001F9288E08F9385E294E09F938F930E94D5
:103FE0004F070F900F900F900F900F900F9096C06B
:103FF00089E295E00E94B6068091D602882309F4F2
:10400000AAC01092D6021092D5021092D402109239
:10401000D3021092D202B1C08BE195E00E94B606A5
:104020000E947F1F7BC08D518093D602833031F177
:1040300070F48130D1F0823009F03FC08AE091E025
:104040009093D5028093D4028BE991E01FC0853014
:1040500059F108F1863089F584E091E09093D5021A
:104060008093D40286ED91E011C08BE091E09093B3
:10407000D5028093D40282E991E008C089E091E002
:104080009093D5028093D40287EA91E09093D30273
:104090008093D20218C088E091E09093D50280937B
:1040A000D40284EB91E0F2CF85E091E09093D502C9
:1040B0008093D40283EC91E0E9CF1092D60288E19C
:1040C00095E00E94B6068091D602882309F455C077
:1040D0001F928F9384E195E00DC08AE015C087E0C0
:1040E00095E01AC097FF47C0108280811F928F937E
:1040F00081E095E09F938F930E944F070F900F9060
:104100000F900F900BC081E0E091D402F091D502A6
:10411000309729F58EEF94E00E94B6062091D602E2
:10412000222359F18091D2029091D302009711F489
:104130008EE891E09F938F931F922F9385EF94E0E9
:104140009F938F930E944F070F900F900F900F90A7
:104150000F900F9016C080E0089586EFD5CF208194
:10416000082E000C990B820F911D8F3F910509F0CD
:104170000CF4B8CF8FEF8083B8CF81EF94E00E942A
:10418000B60681E00895CF93C82F1F928F9382E4E3
:1041900095E09F938F930E944F0781E090E0A0E00D
:1041A000B0E0BC01CD0104C0660F771F881F991FC6
:1041B000CA95D2F70E94340D0F900F900F900F9078
:1041C000CF910C94DC0CDF92EF92FF920F931F9330
:1041D000CF93DF93482F50E0FA013597EF33F10585
:1041E00008F05BC1EE59FF4F0C94422E0E943B1326
:1041F0001F928F9384ED99E09F938F930E944F07B6
:104200000E94371383FB992790F91F929F9382FB9B
:10421000992790F91F929F9381FB992790F91F92FC
:104220009F93982F91701F929F931F928F938BE86B
:1042300099E09F938F930E944F070E943F1387FB43
:10424000222720F91F922F9386FB222720F91F9205
:104250002F9385FB222720F91F922F9384FB22277F
:1042600020F91F922F9383FB222720F91F922F936F
:1042700082FB222720F91F922F9391FB222720F9FE
:104280001F922F93292F21701F922F9381FB22279A
:1042900020F91F922F93282F21701F922F939F9305
:1042A0008F9386EA98E09F938F930E944F078DB774
:1042B0009EB788960FB6F8949EBF0FBE8DBF0E9422
:1042C000E31B982F9695969596951F929F93982FFE
:1042D00091701F929F931F928F9383E798E09F9313
:1042E0008F930E944F078DB79EB708960FB6F8942C
:1042F0009EBF0FBE8DBF06C084E99AE00E94B6063D
:104300000E94D413C1E0CEC081EC96E074C08091CD
:10431000C102817F8E7F8093C1028AE996E00E946C
:10432000B60680E99AE00E94B60681E08093D70243
:10433000E9CF84E79AE00E94B6060E94AF07E2CF79
:104340008091C102C82FC095C170C0FB80F98093D5
:10435000C102CC2319F088E69AE091C08BE59AE07F
:104360000E94B6068091C102897F877F8093C10237
:10437000C9CF9091C10291FBCC27C0F981E0C82739
:10438000892FC0FB81F98093C102CC2319F08EE400
:104390009AE027C080E49AE02EC09091C10292FB7F
:1043A000CC27C0F981E0C827892FC0FB82F9809310
:1043B000C102CC2319F081E39AE013C081E29AE0B4
:1043C0001AC09091C10293FBCC27C0F981E0C827A5
:1043D000892FC0FB83F98093C102CC2351F085E182
:1043E0009AE00E94B6068091C10281608093C1026A
:1043F00059C088E09AE00E94B60684CF8BEC95E025
:10440000FACF0E94D925062FF72EE82ED92EC0917B
:104410000C03C7FBCC27C0F910910B03D0911801F6
:104420000E94B623DF92EF92FF920F931F92CF93D9
:104430001F921F931F92DF931F928F9387E495E043
:104440009F938F930E944F078DB79EB70E960FB61E
:10445000F8949EBF0FBE8DBF55CF0E94DC0C90918B
:104460000C0397FBCC27C0F981E0C827892FC0FB3C
:1044700087F980930C03CC2329F08EEF99E00E94FA
:10448000B60610C083EF99E0B6CF895303C08D51B3
:1044900001C080E00E94C32035CF81EF99E00E94E7
:1044A000B606C0E08C2FDF91CF911F910F91FF9046
:1044B000EF90DF90089580E008950C945B22CF93F5
:1044C000C82F8091D702813071F040F0823009F01E
:1044D00045C08C2F0E94A61F81E046C00E942F126B
:1044E0008232F1F504C00E942F12823261F48C2FC7
:1044F0000E945D22811104C08C2F0E94E3202CC0F9
:1045000081E090E029C08C2F0E945B22811123C0A2
:10451000C431C9F058F4CB3069F0C031B9F482E04D
:104520008093D70288E30E94A61F15C0C93259F0B4
:10453000C83361F48AE996E00E94B6068EE395E0FE
:104540000E94B60608C01092D7020CC08CE395E01A
:104550000E94B60607C081E0817006C01092D702A3
:1045600080E002C080E0F8CFCF910895CF93DF9331
:1045700086319C4541F5EB010E942F12982F8A81CC
:104580002091020130910301882379F09A7A81E029
:1045900009F480E08093D802911102C069E201C061
:1045A00065E3C9010E9409250AC08091D8028111E2
:1045B00002C069E201C065E3C9010E9414250E949E
:1045C000711280E001C081E0DF91CF9108950F93D7
:1045D0001F93CF93DF93C42FD22FFC0182818823B6
:1045E000C9F04093DB020E94CD259093DA028093BC
:1045F000D90280E28C0F883008F057C0C77081E084
:1046000001C0880FCA95EAF7DF91CF911F910F91F2
:104610000C94390A8091DB02481330C08091D90292
:104620009091DA020E94E5258F3A910538F510E263
:104630001D0FCD17B9F080E28C0F883040F4C770A1
:1046400081E001C0880FCA95EAF70E94400A18303D
:1046500028F581E09D2F977001C0880F9A95EAF7A1
:104660000E94390A802F0E94300A1830F0F4D77067
:1046700081E001C0880FDA95EAF70AC080E28C0F6A
:10468000883098F4C77081E001C0880FCA95EAF7B6
:10469000DF91CF911F910F910C94400A802FDF91F1
:1046A000CF911F910F910C94300ADF91CF911F9100
:1046B0000F9108950F939C01CB01243F4CE53407E3
:1046C00031F188F4293DFCE53F07D9F02A3D4CE55E
:1046D000340779F1283D3C45A9F506E221EE41EE8B
:1046E00068ED7CE52BC0263FFCE53F07E1F0A8F034
:1046F000273F3C4539F507E225EE46EE67EF7CE5BE
:104700001DC007E225EE45EE69ED7CE517C006E227
:1047100021EE40EE64EF7CE511C007E225EE44EEA9
:1047200065EF7CE50BC006E221EE42EE66EF7CE52C
:1047300005C008E221E045EE6AED7CE50E94E72233
:1047400080E008C0FC018281882319F01092DB020E
:1047500001C081E00F9108959093FB018093FA01CD
:1047600008959093E1028093E0020895E091E002C1
:10477000F091E102309721F00190F081E02D099451
:1047800080E00895EF92FF921F93CF93DF93FC0197
:10479000A091E002B091E102109709F442C080912B
:1047A0001801882341F080910C0387FF04C08081A9
:1047B000818386E08083EF011296ED91FC9113973F
:1047C000CE0109958091C10282FF2BC080FF04C0F9
:1047D0008DEA9AE00E94B60618E087EAE82E8AE0A1
:1047E000F82E8091C10280FF0BC088811F928F93A9
:1047F000FF92EF920E944F070F900F900F900F9033
:10480000115021961111EDCF8091C10280FF09C096
:1048100085EA9AE0DF91CF911F91FF90EF900C9481
:10482000B606DF91CF911F91FF90EF900895E09130
:10483000E002F091E102309739F022E0DC012C93A4
:104840000480F581E02D099408952091DE023091D5
:10485000DF022817390771F09093DF028093DE02A0
:10486000E091E002F091E102309721F00680F781BB
:10487000E02D099408952091DC023091DD02281783
:10488000390771F09093DD028093DC02E091E00241
:10489000F091E102309721F00084F185E02D099438
:1048A0000895FC01329680911801882331F080919F
:1048B0000C0387FF02C09EE101C096E080E09150AA
:1048C00028F021912223D9F38F5FF9CF0895662331
:1048D00051F1209118012223E9F020910C0327FFC8
:1048E00019C0462F4695469546954E31E0F46770BF
:1048F00021E030E002C0220F331F6A95E2F7FC018D
:10490000E40FF11D828190E02823392381E0232BDD
:1049100069F409C0FC01329608962191621729F0CA
:10492000E817F907D1F780E0089581E008959C0128
:10493000FC0132969FEF80E04191461789F09F3F3E
:1049400019F4411101C0982F8F5F8630A9F79F3F5E
:1049500039F0F901E90FF11D97FDFA956283089589
:1049600008959C012A5F3F4FFC014281461301C01C
:104970001282019682179307B9F70895262F26957C
:10498000269526952E3170F4FC01E20FF11D67701B
:1049900021E030E001C0220F6A95EAF78281282BDE
:1049A000228308958091C10280FF0CC01F926F93F3
:1049B0008DED9AE09F938F930E944F070F900F9079
:1049C0000F900F900895262F2695269526952E3127
:1049D00078F4FC01E20FF11D677021E030E001C0C6
:1049E000220F6A95EAF72095828128232283089571
:1049F0008091C10280FF0CC01F926F938FEB9AE0F1
:104A00009F938F930E944F070F900F900F900F90DE
:104A1000089520911801222329F020910C0327FDED
:104A20000C94BE240C94972420911801222329F081
:104A300020910C0327FD0C94E3240C94B1242091C5
:104A40001801FC013296222331F080910C0387FF7C
:104A500002C08EE101C086E0DF011D928A95E9F770
:104A6000089508950C94312583E08093E2020C941C
:104A70003225811102C081E001C082E08093E20210
:104A80000C9432250C94392581E08093E2020C9439
:104A900032250C94442508950C944B250C944C25F8
:104AA0000C944B250C944B250C944B25CF930E94D2
:104AB00052250E942F180E945025C0E08C2F0E9482
:104AC0000417892B29F4CF5FC530C1F780E001C0FE
:104AD00081E0CF91089508951F920F920FB60F9223
:104AE00011248F939F93AF93BF938091E302811121
:104AF00013C08091230390912403A0912503B091CA
:104B000026034196A11DB11D809323039093240396
:104B1000A0932503B0932603BF91AF919F918F91EE
:104B20000F900FBE0F901F90189580912B0384302B
:104B300031F10E9436081092E30220E488E190E00F
:104B40000FB6F894A895809360000FBE2093600084
:104B500083B7817F846083BF83B7816083BF78948C
:104B6000889583B78E7F83BF0FB6F894A895809100
:104B70006000886180936000109260000FBE08950D
:104B80000E94DC0C0C943D0882E084BD93E095BD4E
:104B90009AEF97BD80936E0008952FB7F894809197
:104BA000230390912403A0912503B09126032FBFE6
:104BB00008952FB7F8946091230370912403809196
:104BC0002503909126032FBF08959C014FB7F894B9
:104BD0008091230390912403A0912503B091260393
:104BE0004FBF821B930B089578941F920F920FB6BC
:104BF0000F9211248F939F93AF93BF9380912303C0
:104C000090912403A0912503B09126030196A11D44
:104C1000B11D8093230390932403A0932503B093A5
:104C20002603BF91AF919F918F910F900FBE0F9070
:104C30001F90189581E08093E00080E28093D80077
:104C40001092C9008FE19EE40197F1F700C00000C7
:104C500087E090EBDC018093340390933503A093BD
:104C60003603B09337039CE088E10FB6F894A8951B
:104C7000809360000FBE90936000FFCF80910A0385
:104C80000895089522E02093E9002FEF3091E80085
:104C9000215035FD06C035ED3A95F1F700002111A0
:104CA000F5CF2091E80025FF0BC040E050E066E022
:104CB00070E00E943F298091E8008E778093E800A1
:104CC0000895CF93DF9320911801222339F020918A
:104CD0000C0327FF03C060E222E002C068E021E08D
:104CE0002093E9002FEF3091E800215035FD06C0F8
:104CF00035ED3A95F1F700002111F5CF2091E8004C
:104D000025FF1DC0EC0180911801811105C040E014
:104D100050E068E070E003C070E040E050E0CE0199
:104D20000E943F298091E8008E778093E80080E21E
:104D3000FE01AAEEB2E001900D928A95E1F7DF91B3
:104D4000CF9108958093E6027093E8026093E702A2
:104D500080912B03843001F582E08093E9008FEF8E
:104D60009091E800815095FD06C095ED9A95F1F778
:104D700000008111F5CF8091E80085FF0DC040E073
:104D800050E063E070E086EE92E00E943F2980915F
:104D9000E8008E778093E8000895BC0184E00C94CD
:104DA000A226BC0183E00C94A2268FE09BE00E9427
:104DB000B60680912A03811109C00E94D02A0E9460
:104DC0002D2B8091E20084608093E20008958BE0B7
:104DD0009BE00E94B60610922A03089587E09BE0AC
:104DE0000E94B6060C94492583E09BE00E94B6061B
:104DF0006091270381E0611101C080E00C943425AB
:104E00008FEF9AE00E94B60690912B0381E09430D8
:104E100009F080E0609127030C9439252091E50288
:104E20002F5F822F62E30E94EC2D992319F02093CB
:104E3000E50208951092E5028091E902882371F15C
:104E400080912B03843041F58091E9008F7020918F
:104E5000EC00922F917020FD90E8892B93E09093C5
:104E6000E9009091EB0090FF14C09091EE0097FF45
:104E700010C09091E80095FF03C01092F100F9CFA7
:104E80009091E80090FF05C09091E8009E77909384
:104E9000E8008F708093E9001092E902089542E0E3
:104EA00061EC81E00E94492A42E261EC82E00E94CA
:104EB000492A42E261EC83E00E94492A90912B0347
:104EC00081E0943009F080E0609127030C94422542
:104ED00080912D03833009F461C030F4813071F08A
:104EE000823009F49AC008958A3009F486C08B3064
:104EF00009F46CC0893009F0A8C020C080912C034F
:104F0000813A09F0A2C08091E800877F8093E80091
:104F10008091300390913103892B21F460E28AEE75
:104F200092E003C060E080E090E070E00E948A2997
:104F30008091E8008B778093E800089580912C039E
:104F4000813209F082C08091300390913103029741
:104F500008F07BC08091E800877F8093E800809113
:104F6000E80082FD05C080912B038111F8CF6DC050
:104F70002091F3008091F20090E0922B029731F49F
:104F80008091F100813011F0863021F48091F100A0
:104F900080930A038091E8008B7753C080912C03A3
:104FA000813A09F052C08091300390913103892BEE
:104FB00009F04BC08091E800877F8093E8008091E2
:104FC000E80080FFFCCF8091180136C080912C034F
:104FD0008132D9F58091300390913103892BA9F565
:104FE0008091E800877F8093E8000E947E2A80916C
:104FF0002E03809318010C94DC0C80912C038132D9
:1050000021F58091E800877F8093E8000E947E2A46
:1050100080912F0380930B03089580912C03813A94
:10502000A1F48091E800877F8093E8008091E800F8
:1050300080FFFCCF80910B038093F1008091E8000A
:105040008E778093E8000C947E2A08959FB7F89499
:105050001092E9029FBF90912B03943009F057C042
:105060009091E9009F703091EC00232F217030FD6A
:1050700020E8922B23E02093E9002091EB0020FF11
:1050800043C02091EE0027FF3FC02091E40222237D
:1050900021F02091E80025FF37C01092E40226E0BD
:1050A0003091E80035FD15C030912B03343061F5A7
:1050B0003091EB0035FD28C0215021F481E0809330
:1050C000E40222C0EFE9FFE03197F1F700C00000F1
:1050D000E7CF8093F1008091E80085FD0AC08091C0
:1050E000E80080FFFCCF8091E8008E778093E80095
:1050F00006C08FB7F89421E02093E9028FBF9F701C
:105100009093E90080E008959F709093E9008FEFFD
:10511000089584B7877F84BF0FB6F894A8958091CF
:105120006000886180936000109260000FBE90E084
:1051300080E80FB6F89480936100909361000FBEF1
:105140000C9444250E94D02A0E942D2BE2EEF0E020
:1051500080818460808378940C94C12D8CE091E0F0
:105160000C94B12380912B038530C9F48BEF9AE026
:105170000E94B60680912B03853079F40E94952514
:10518000809129038823B1F30E945625882391F347
:105190000E9429290E94DC0CEDCF0C94C0250895B3
:1051A00008950C94D328292F332723303105C9F0D3
:1051B00060F42130310581F02230310509F041C021
:1051C0008BE590E02BE53BE040C021323105E1F07A
:1051D0002232310531F135C082E190E026EB3BE02F
:1051E00034C099278130910549F028F0029749F59C
:1051F000E3E1FBE005C0E7E5FBE002C0E3E3FBE041
:10520000849190E09F0121C063307105D0F4660F56
:10521000771FFB01EC50FE4F2081318189E090E047
:1052200014C06330710568F4FB01EE0FFF1FE251FB
:10523000FE4F20813181FB01E551FE4F808190E0DE
:1052400004C080E090E020E030E0FA013183208368
:10525000089580E189BD82E189BD09B400FEFDCFDA
:105260008091D8008F7D8093D8008091E00082608B
:105270008093E0008091E00081FDFCCF0895CF9203
:10528000DF92EF92FF920F931F93CF93DF93EC0186
:105290008B017A010E949D2A811133C0E114F1042F
:1052A00039F0F70180819181081B190BC80FD91FB4
:1052B000C12CD12C0115110519F18091E80085FD53
:1052C00016C08091E8008E778093E800E114F10425
:1052D00049F0F70180819181C80ED91ED182C08228
:1052E00085E00FC00E949D2A882321F30AC089917E
:1052F0008093F10001501109FFEFCF1ADF0ADACFD6
:1053000080E0DF91CF911F910F91FF90EF90DF90A0
:10531000CF90089520913203309133032617370739
:1053200048F06115710539F42091E8002E7720933B
:10533000E80001C0B901FC0120E06115710579F1B7
:1053400080912B038823F1F18530F1F18091E80001
:1053500083FD3CC08091E80082FD2EC08091E80072
:1053600080FFEBCF2091F3008091F20090E0922B30
:105370006115710551F08830910538F42191209321
:10538000F100615071090196F3CF21E0089709F00F
:1053900020E08091E8008E778093E800CECF211145
:1053A000CFCF0AC080912B03882361F0853061F054
:1053B0008091E80083FD0AC08091E80082FFF2CF6F
:1053C00080E0089582E0089583E0089581E00895E3
:1053D00020913203309133032617370748F06115C7
:1053E000710539F42091E8002E772093E80001C080
:1053F000B901FC0120E06115710591F180912B0349
:10540000882309F440C0853009F43FC08091E8004A
:1054100083FD3DC08091E80082FD2FC08091E800AF
:1054200080FFE9CF2091F3008091F20090E0922B71
:105430006115710559F08830910540F4249120934D
:10544000F1003196615071090196F2CF21E0089781
:1054500009F020E08091E8008E778093E800CBCFC0
:105460002111CCCF0AC080912B03882361F08530B5
:1054700061F08091E80083FD0AC08091E80082FF1E
:10548000F2CF80E0089582E0089583E0089581E0FE
:105490000895982F973068F59093E900981739F0A0
:1054A0007091EC002091ED005091F00003C0242F8A
:1054B000762F50E021FD02C09F5FECCF3091EB00D2
:1054C0003E7F3093EB003091ED003D7F3093ED0057
:1054D0003091EB0031603093EB007093EC0020933F
:1054E000ED005093F0002091EE0027FDE5CF80E025
:1054F00008958F708093E90081E0089580912C03D6
:1055000087FF11C08091E80082FD05C080912B03C8
:105510008111F8CF11C08091E8008B770BC080918A
:105520002B03882349F08091E80080FFF8CF809119
:10553000E8008E778093E80008952091E400309190
:10554000E50095E64091EC00842F817040FF23C078
:105550008091E80080FD1DC080912B03882399F085
:10556000853099F08091EB0085FD11C04091E400F9
:105570005091E5002417350729F3915011F09A0155
:10558000E1CF84E0089582E0089583E0089581E00A
:10559000089580E008954091E80042FFDDCF08952E
:1055A0000E943E2B0E94462BE0EEF0E0808181605D
:1055B0008083E8EDF0E080818F77808319BCA7EDD0
:1055C000B0E08C918E7F8C9380818F7E808310924F
:1055D0002A0308950F931F93CF93DF930E943E2BCE
:1055E0000E94462BC8EDD0E088818F778883888120
:1055F0008068888388818F7D888319BC10922B03F3
:1056000010922703109229031092280300EE10E055
:10561000F80180818B7F808388818160888342E06C
:1056200060E080E00E94492AE1EEF0E080818E7F18
:105630008083E2EEF0E080818160808380818860F9
:105640008083F80180818E7F808388818061888358
:10565000DF91CF911F910F910895E8EDF0E08081E7
:105660008F7E8083E7EDF0E080818160808384E03D
:1056700082BF81E080932A030C94EA2AE8EDF0E0EF
:1056800080818E7F80831092E20008951092DA006C
:105690001092E10008951F920F920FB60F921124FD
:1056A0002F933F934F935F936F937F938F939F932A
:1056B000AF93BF93EF93FF938091E10082FF0BC004
:1056C0008091E20082FF07C08091E1008B7F809390
:1056D000E1000E940E278091DA0080FF1FC08091B8
:1056E000D80080FF1BC08091DA008E7F8093DA00A3
:1056F0008091D90080FF0DC080E189BD82E189BD24
:1057000009B400FEFDCF81E080932B030E94D526D3
:1057100005C019BC10922B030E94E7268091E1007E
:1057200080FF19C08091E20080FF15C08091E200E7
:105730008E7F8093E2008091E20080618093E2009E
:105740008091D80080628093D80019BC85E0809356
:105750002B030E94F4268091E10084FF30C08091E9
:10576000E20084FF2CC080E189BD82E189BD09B4DB
:1057700000FEFDCF8091D8008F7D8093D80080916E
:10578000E1008F7E8093E1008091E2008F7E809324
:10579000E2008091E20081608093E2008091270323
:1057A000882311F084E007C08091E30087FD02C0E8
:1057B00081E001C083E080932B030E940027809149
:1057C000E10083FF29C08091E20083FF25C0809122
:1057D000E100877F8093E10082E080932B031092A9
:1057E00027038091E1008E7F8093E1008091E200A9
:1057F0008E7F8093E2008091E20080618093E200DE
:1058000042E060E080E00E94492A8091F0008860D8
:105810008093F0000E94EE26FF91EF91BF91AF912F
:105820009F918F917F916F915F914F913F912F91B8
:105830000F900FBE0F901F9018951F920F920FB6EA
:105840000F9211242F933F934F935F936F937F9306
:105850008F939F93AF93BF93CF93DF93EF93FF9378
:10586000C091E900CF708091EC00D82FD17080FDFD
:10587000D0E81092E9008091F000877F8093F000DB
:1058800078940E94612C1092E9008091F000886069
:105890008093F000CD2BCF70C093E900FF91EF9182
:1058A000DF91CF91BF91AF919F918F917F916F9138
:1058B0005F914F913F912F910F900FBE0F901F90CE
:1058C00018951F93CF93DF93CDB7DEB7AA970FB686
:1058D000F894DEBF0FBECDBFECE2F3E08091F100A3
:1058E000819323E0E433F207C9F70E94682780918F
:1058F000E80083FF2EC180912C0390912D03492F46
:1059000050E04A30510508F024C1FA01EF55FF4F2D
:105910000C94422E803821F0823809F01AC108C058
:105920008091280390912903992389F082600FC008
:10593000809130038F70873008F00BC18093E900AD
:105940008091EB0085FB882780F91092E900909107
:10595000E800977F9093E8008093F1001092F100A7
:10596000D1C0282F2D7F09F0F4C0882319F0823090
:1059700061F0EFC080912E03813009F0EAC09330CE
:1059800009F080E0809329032EC080912E038111BD
:105990002AC0809130038F702FEF280F263008F037
:1059A000D8C08093E9002091EB0020FF1CC0933009
:1059B00021F48091EB00806214C09091EB00906123
:1059C0009093EB0021E030E0A90102C0440F551F85
:1059D0008A95E2F74093EA001092EA008091EB008A
:1059E00088608093EB001092E9008091E800877F47
:1059F0008093E8000E947E2AACC08111AAC0109159
:105A00002E031F778091E3008078812B8093E30041
:105A10008091E800877F8093E8000E947E2A809131
:105A2000E80080FFFCCF8091E30080688093E30072
:105A3000111102C082E001C083E080932B0389C072
:105A40008058823008F085C080912E0390912F03FA
:105A50008C3D53E0950779F583E08A838AE2898358
:105A60004FB7F894DE01139620E03EE051E2E32FB9
:105A7000F0E050935700E49120FF03C0E295EF70EF
:105A80003F5FEF708E2F90E0EA3010F0C79601C0B4
:105A9000C0968D939D932F5F243149F74FBF80911E
:105AA000E800877F8093E8006AE270E0CE0101960B
:105AB0000E948A2916C06091300370913103AE01B3
:105AC0004F5F5F4F0E94D128BC01892B09F441C070
:105AD0009091E800977F9093E80089819A810E94D5
:105AE000E8298091E8008B778093E80032C0803805
:105AF00081F58091E800877F8093E80080912703FB
:105B00008093F1008091E8008E7772CF811121C0DF
:105B100080912E0390912F0399270297D4F48091BE
:105B2000E800877F8093E80080912E03809327030D
:105B30000E947E2A80912703811106C08091E30094
:105B400087FD02C081E001C084E080932B030E94A6
:105B50004F278091E80083FF0AC08091E800877F8B
:105B60008093E8008091EB0080628093EB00AA961E
:105B70000FB6F894DEBF0FBECDBFDF91CF911F915E
:105B80000895CF9380912B038823A1F0C091E90061
:105B9000CF709091EC00892F817090FD80E8C82B28
:105BA0001092E9008091E80083FD0E94612CCF7083
:105BB000C093E900CF910895DB018F939F930E94DA
:105BC000572EBF91AF91A29F800D911DA39F900D65
:105BD000B29F900D11240895991B79E004C0991F7C
:105BE000961708F0961B881F7A95C9F78095089537
:105BF000AA1BBB1B51E107C0AA1FBB1FA617B707F3
:105C000010F0A61BB70B881F991F5A95A9F780950E
:105C10009095BC01CD01089597FB072E16F40094D2
:105C200007D077FD09D00E94F82D07FC05D03EF47F
:105C3000909581959F4F0895709561957F4F089538
:105C4000A1E21A2EAA1BBB1BFD010DC0AA1FBB1F80
:105C5000EE1FFF1FA217B307E407F50720F0A21BF2
:105C6000B30BE40BF50B661F771F881F991F1A945F
:105C700069F760957095809590959B01AC01BD0189
:105C8000CF010895EE0FFF1F0590F491E02D0994C8
:105C9000A29FB001B39FC001A39F700D811D11246D
:105CA000911DB29F700D811D1124911D08950E94B8
:105CB000482EA59F900DB49F900DA49F800D911D1F
:105CC00011240895FB01DC0104C08D91019080191D
:105CD00021F441505040C8F7881B990B0895F99959
:105CE000FECF92BD81BDF89A992780B50895A8E1AD
:105CF000B0E042E050E00C94A32E262FF999FECF9D
:105D000092BD81BDF89A019700B4021639F01FBA0E
:105D100020BD0FB6F894FA9AF99A0FBE089503962B
:105D2000272F0E947E2E0E947D2E252F0E947E2EE0
:105D3000242F0C947E2E0196272F0E947E2E0C94E9
:105D40007D2EDC01CB01FC01F999FECF06C0F2BD2E
:105D5000E1BDF89A319600B40D9241505040B8F729
:065D60000895F894FFCF46
:105D6600AF008D02280850011E0A14013E26612646
:105D76004226D126CD26412601E200E900EA00B5F9
:105D860000B600B700CD008301CC008A01920194D1
:105D9600012102230224022502260227022A02B337
:105DA60000B4006F007000818283E200E900EA001F
:105DB600B500B600B700CD008301CC008A01920180
:105DC60094012102230224022502260227022A0226
:105DD600B300B4006F007000818283F531F0F1F4F6
:105DE60033979694959392919030323435363F3F5F
:105DF6003F006D6B5F64656C6179006D6B5F696E0A
:105E060074657276616C006D6B5F6D61785F73703F
:105E1600656564006D6B5F74696D655F746F5F6D5A
:105E26006178006D6B5F776865656C5F6D61785F43
:105E36007370656564006D6B5F776865656C5F742C
:105E4600696D655F746F5F6D61780040B622A00C66
:0A5E5600EA0BC80B6D0B860B9F0BC7
:00000001FF
